:04000000B6017429A8
:100008000800B616B61EB612B6190E28B615472041
:10001800031835280830A3005B20A20DA30B102875
:10002800B61E402065206120B61A35203A202208E5
:1000380003106F29B616B61EB61236192828FE39CF
:10004800B700361503106F29361A3028A600361661
:1000580047200318352826084E2003183528B61ED1
:100068006F294020652036113612B6113A088400EF
:1000780038088417800446283A088400380980051F
:100088008417800508003A20652040206120370841
:10009800B6190138A2000830A300A20D03183A20AF
:1000A800031C402065206120A30B51283A206520BD
:1000B8003A08840038080005FF3E3B0884003909E7
:1000C80043283B08840039083D282C08A0002D0847
:1000D800A1000130A20064009520031C8228A20B15
:1000E8006F28FF30A007031CA107031C6F29FA30F3
:1000F800A2006F286400952003187E28E720A80135
:100108000830A300E82095200318A80AAB1EA80110
:10011800A20CA30B8628AB1AA213E820031422080A
:1001280008003A08840038088417800484130005FE
:100138002B1B3806FF3E0800A400290803140319E6
:100148006F296A21031C0800A000251883172408BA
:100158008400200880008313A40AA903A1280408A6
:10016800A6003A088400F030B7050830A70003104D
:100178000318B70ACD20A60CA70BBC280000AB1AA1
:10018800370CCD2072210314CD202F08A3002E0890
:1001980006298413AB1FDC28000838042B1F3806F7
:1001A8008000841700083804031C38068000E828FB
:1001B80000083804031C38062B1B380680008417F7
:1001C80038098005E82837172B081F39003EA10099
:1001D8002A080E3E0318A10A371F13293713A00057
:1001E800023025211329A400290803196F2925188D
:1001F800831724088400000883136A21A40AA9032A
:10020800F828A301A200FF30A207031CA307031CC0
:100218006F290330A100E73013210729A101FC3E13
:10022800A000A109031C1E29FF300000A007031825
:100238001929A0076400A10F182908000310A10CB0
:10024800A00CFF3E0318222920086F29A101A30151
:10025800A20002303929A101A301A20001303929E5
:10026800A101A301A20004303929A8002308210212
:10027800031D402922082002043003180130031905
:1002880002302805031DFF306F290038031DFF3099
:100298000405031DFF306F290404031DFF306F2977
:1002A8001030A800A101A001A70CA60C031C62290C
:1002B8002208A00723080318230FA107A10CA00CEC
:1002C800A50CA40CA80B582924086F298400310810
:1002D8008A00300882008313031383126400080025
:1002E800831607309F008312BC01BD018316861652
:1002F8000617861706108610061186110612880141
:100308000710871007118711071287128312CE0171
:10031800C4018801C901CB01CC01C701CD01880105
:1003280087100711071086140611CF01C60187161A
:1003380064308A01052187120A308A01052187164F
:100348000230A30058308A0106218A110A12342F7C
:10035800071406308A011221071008008710861436
:1003680006110130C9006400033049028A110A12DB
:100378000318E0293E308800C03088008A01AC218B
:10038800403088008A01AC21B83088008A01AC214D
:100398003F3088008A01AC2183108618831406191F
:1003A8008614061D861083180615831C0611C90AB3
:1003B8008A110A12031DB72986140611080087102E
:1003C8003E3088008A01AC21861406110130C9002C
:1003D8006400033049028A110A1203182E2AB83021
:1003E800CB006400C0304B028A110A1203181E2A7F
:1003F80087108A01AC21403088008A01AC214B0863
:1004080088008A01AC2187140130CC006400413097
:100418004C028A110A120318192A88018A01AC2190
:10042800CC0A8A110A12031D0A2ACB0A8A110A1257
:10043800031DF52983108618831406198614061DD2
:10044800861083180615831C0611C90A8A110A1218
:10045800031DEC29861006158710B83088008A011C
:10046800AC21C03088008A01AC21403088008A0164
:10047800AC2186140611B83088008A01AC21C0303E
:1004880088008A01AC21403088008A01AC213F30C5
:1004980088008A01AC218714861406110800871485
:1004A800DF304407B200FF300318013EB3003208C2
:1004B800A6003308A7000530A200A3018A01542131
:1004C800BE002508BF0004303E07C0003F080318DF
:1004D800013EC1003E08BC003F08BD003C08A0002A
:1004E8003D08A1004108A30040088A0131218A1172
:1004F8000A12031DA02A8A110A12AC220730BA0078
:100508001030B8000730BB000830B900A0308A01AD
:1005180020203D088A0120203C088A0120208A01E9
:10052800052088008A01AC21C70ABC0A0319BD0A44
:100538008A110A12031D722A8A110A12A4220800BB
:100548008A110A12AC2288018A01AC21C70A080064
:1005580064004708403C8A110A12031DBB2A861012
:1005680006158710403088008A01AC218714640082
:100578004708803C8A110A12031DCC2A86140611EA
:10058800CD0AC7018710403088008A01AC21871442
:1005980064004D08083C8A110A12031DDD2ACD01AA
:1005A80064005008013C8A110A12031DDD2A073035
:1005B800CD008710B8304D0788008A01AC21871418
:1005C800080064003F3047028A110A120318F32A10
:1005D800861406114708C6008A110A12F82A8610DE
:1005E800061540304702C6008710B8304D0788000E
:1005F8008A01AC214030460788008A01AC21871463
:1006080008000830C700CD018A01E522C90164004D
:10061800143049028A110A120318582B4908133C4E
:100628008A110A12031C372B8A110A121F23C400CD
:100638008A110A12372B03308A0049088207473487
:1006480072346134703468346934633420344C341F
:100658004334443420345434653472346D3469344A
:100668006E3461346C3464004408203C8A110A12E8
:10067800031D512B0130CB00640004304B028A115A
:100688000A1203184E2B8A01A422CB0A8A110A12D5
:10069800031D402B8A110A12532B8A015322C90ABF
:1006A8008A110A12031D0B2B0130CB0064000530A0
:1006B8004B028A110A120318922BC7014B08CD006E
:1006C8008A01E522C9016400403049028A110A12F0
:1006D8000318772B143088008A01AC21C90A8A11C3
:1006E8000A12031D672B4030C7008A01E522C901A1
:1006F8006400803049028A110A1203188C2B1430C6
:1007080088008A01AC21C90A8A110A12031D7C2BB0
:100718000330CB078A110A12031C5A2BC701053074
:10072800CD008A01E522C9016400173049028A1107
:100738000A120318E82B4908163C8A110A12031CEE
:10074800C72B8A110A12AC23C4008A110A12C72BBC
:1007580003308A0049088207533465346E346434A0
:10076800203463346D346434733420346F346E341D
:100778002034613420347434653472346D3469340F
:100788006E3461346C3464004408203C8A110A12C7
:10079800031DE12B0130CB00640004304B028A11A9
:1007A8000A120318DE2B8A01A422CB0A8A110A1224
:1007B800031DD02B8A110A12E32B8A015322C90A7E
:1007C8008A110A12031D982BC7010630CD008A0131
:1007D800E522C9016400403049028A110A1203184F
:1007E800FE2B3C3088008A01AC21C90A8A110A1202
:1007F800031DEE2B4030C7008A01E522C9016400C1
:10080800803049028A110A120318132C3C308800E0
:100818008A01AC21C90A8A110A12031D032CC701D7
:100828000230CD008A01E522C90164000A3049027C
:100838008A110A1203185C2C4908093C8A110A1209
:10084800031C3B2C8A110A122D24C4008A110A1297
:100858003B2C04308A004908820750346F347234C4
:10086800743442342034503469346E347334640040
:100878004408203C8A110A12031D552C0130CB0074
:10088800640004304B028A110A120318522C8A01A0
:10089800A422CB0A8A110A12031D442C8A110A12B7
:1008A800572C8A015322C90A8A110A12031D192CCE
:1008B8004030C7000230CD008A01E522C90164003A
:1008C8000B3049028A110A120318A72C49080A3C5E
:1008D8008A110A12031C862C8A110A127724C40072
:1008E8008A110A12862C04308A004908820750347B
:1008F8006F34723474344334203453347434613470
:100908007434653464004408203C8A110A12031DBB
:10091800A02C0130CB00640004304B028A110A126B
:1009280003189D2C8A01A422CB0A8A110A12031DDE
:100938008F2C8A110A12A22C8A015322C90A8A1101
:100948000A12031D632C0800861006150130C90021
:100958006400033049028A110A120318DD2C87103B
:10096800BF3088008A01AC21403088008A01AC2160
:100978008714CB01640041304B028A110A12031814
:10098800CD2C88018A01AC21CB0A8A110A12031DD9
:10099800BE2C83108618831406198614061D86102B
:1009A80083180615831C0611C90A8A110A12031D29
:1009B800AC2C86140611C7010730CD000800420888
:1009C800A00042308A012A21B2004208A000623009
:1009D8008A012A21B4003208840034088A0150218F
:1009E800B400B5006400340835048A110A120319EA
:1009F800142E30304302C80064004808003C8A11B5
:100A08000A12031D292D013086068316061083124B
:100A18004D08D1004708D2000330CD00C7018A0134
:100A2800E52264008A110A12061C1F2D3130C40009
:100A38008A110A12212D3030C4008A01532251082C
:100A4800CD005208C7008A01E52264004808033C2B
:100A58008A110A12031D582D08308606831686113E
:100A68000130831286068316061083124D08D100C2
:100A78004708D2000330CD000830C7008A01E522BC
:100A880064008A110A12861D4E2D3130C4008A1165
:100A98000A12502D3030C4008A0153225108CD006B
:100AA8005208C7008A01E52264004808043C8A11FC
:100AB8000A12031D872D1030860683160612013090
:100AC800831286068316061083124D08D100470844
:100AD800D2000330CD001230C7008A01E52264003D
:100AE8008A110A12061E7D2D3130C4008A110A129D
:100AF8007F2D3030C4008A0153225108CD0052089E
:100B0800C7008A01E52264004808053C8A110A12D8
:100B1800031DB62D203086068316861201308312F7
:100B280086068316061083124D08D1004708D200A6
:100B38000330CD001C30C7008A01E52264008A1109
:100B48000A12861EAC2D3130C4008A110A12AE2D4D
:100B58003030C4008A0153225108CD005208C70022
:100B68008A01E52264004808063C8A110A12031D1E
:100B7800E52D40308606831606130130831286065B
:100B88008316061083124D08D1004708D20003309F
:100B9800CD002630C7008A01E52264008A110A12B6
:100BA800061FDB2D3130C4008A110A12DD2D3030CA
:100BB800C4008A0153225108CD005208C7008A0197
:100BC800E52264004808073C8A110A12031D142E06
:100BD80080308606831686130130831286068316B4
:100BE800061083124D08D1004708D2000330CD000B
:100BF8003030C7008A01E52264008A110A12861F74
:100C08000A2E3130C4008A110A120C2E3030C4006A
:100C18008A0153225108CD005208C7008A01E522F3
:100C28004208C40008004D08D1004708D200440813
:100C3800D3000330CD00C7018A01E52264008A1180
:100C48000A12061C2C2E3130C4008A110A122E2ECC
:100C58003030C4008A0153220830C7008A01E522D7
:100C680064008A110A12861D3E2E3130C4008A1192
:100C78000A12402E3030C4008A0153221230C700B5
:100C88008A01E52264008A110A12061E502E3130AC
:100C9800C4008A110A12522E3030C4008A0153222D
:100CA8001C30C7008A01E52264008A110A12861ED8
:100CB800622E3130C4008A110A12642E3030C4000A
:100CC8008A0153222630C7008A01E52264008A116E
:100CD8000A12061F742E3130C4008A110A12762EA9
:100CE8003030C4008A0153223030C7008A01E5221F
:100CF80064008A110A12861F862E3130C4008A11B8
:100D08000A12882E3030C4008A0153225108CD00BF
:100D18005208C7005308C4008A01E52208004D089C
:100D2800D1004708D2004408D3000330CD0040303A
:100D3800C7008A01E52264008A110A12071CA92E3D
:100D48003130C4008A110A12AB2E3030C4008A0137
:100D580053224830C7008A01E52264008A110A122A
:100D6800871CBB2E3130C4008A110A12BD2E3030C8
:100D7800C4008A0153225030C7008A01E52264006A
:100D88008A110A12071DCD2E3130C4008A110A12A9
:100D9800CF2E3030C4008A0153225830C7008A0150
:100DA800E52264008A110A12871DDF2E3130C40043
:100DB8008A110A12E12E3030C4008A0153226030B1
:100DC800C7008A01E52264008A110A12071EF12E63
:100DD8003130C4008A110A12F32E3030C4008A015F
:100DE80053226830C7008A01E52264008A110A127A
:100DF800871E032F3130C4008A110A12052F3030A4
:100E0800C4008A0153227030C7008A01E5226400B9
:100E18008A110A12071F152F3130C4008A110A12CD
:100E2800172F3030C4008A0153227830C7008A0156
:100E3800E52264008A110A12871F272F3130C40067
:100E48008A110A12292F3030C4008A01532251080E
:100E5800CD005208C7005308C4008A01E5220800E3
:100E68008A01B2218A01E3218A0105238A01172612
:100E7800C7010730CD008A01E522861406118710C4
:100E8800403088008A01AC21BF3088008A01AC213B
:100E980087140130D0000730BA004030B800543011
:100EA800AA00AB01AE01AF0152308A01B42045302F
:100EB8008A01B42041308A01B42044308A01B42028
:100EC80059308A01B4203A308A01B4200A308A01A4
:100ED800B4200D308A01B4208A0117268A0193268E
:100EE8000730BA008030B8005430AA00AB01F430A3
:100EF800AC000130AD008A0169208A110A12031C76
:100F0800702FC400640044081B3C8A110A12031D98
:100F1800D32F0730BA004030B8005430AA00AB01D4
:100F2800AE01AF0143308A01B4204D308A01B420AC
:100F380044308A01B4203A308A01B4200730BA001C
:100F48008030B8005430AA00AB018A017E20403CB2
:100F58008A110A12031DA92F0230A9007E30B000A1
:100F6800B101A50142308A01A0200730BA00403003
:100F7800B8005430AA00AB01AE01AF010230A9009D
:100F8800B330B000B101A50142308A01F7200A3020
:100F98008A01B4200D308A01B4208A01E324440870
:100FA800A00008308A012A21B2004F08A0000530AD
:100FB8008A012F21B4003208840034088A014921AB
:100FC800B400B5006400340835048A150A12031900
:100FD80008280630C7020630CF028710403047077E
:100FE80088008A01AC218714C901640006304902CF
:100FF8008A150A120318082888018A01AC21C90A2F
:101008008A110A12031DF92F64004408203C8A152E
:101018000A12031D11288A01A4224408A0002130C5
:101028008A013421B2004408A0007E308A012F21B1
:10103800B400320834048A110A12031D702F8A0181
:1010480053220630CF07640080304F028A150A12F7
:10105800031C31288A01A824CF018A01702F63005C
:061068008A150A1233286C
:02400E00753DFE
:00000001FF
